:020000040003F7
:10AC0000383800200DAD030027AD030029AD030047
:10AC10000000000000000000000000000000000034
:10AC20000000000000000000000000002BAD030049
:10AC300000000000000000002DAD03002FAD030058
:10AC400031AD030031AD030031AD030031AD030080
:10AC500031AD03000000000031AD030031AD030051
:10AC600031AD030031AD030031AD030031AD030060
:10AC700031AD03005DBC030031AD030031AD030015
:10AC800031AD0300BDBC030031AD030031AD0300A5
:10AC9000DDBC030031AD0300E5BC030031AD0300B2
:10ACA00031AD030031AD03000000000000000000E2
:10ACB0000000000000000000000000000000000094
:10ACC0000448854600F080F80048004735D003006E
:10ACD000C046C04638380020056885F308884068BB
:10ACE000FF2464B2EFF30585002D01D1A64600478D
:10ACF0002546064621273FBAF0B400240025002649
:10AD00000027F0B4F92040B20047000003210948B1
:10AD100002680A430260084802680A430260074862
:10AD2000804707480047FEE7FEE7FEE7FEE7FEE74D
:10AD3000FEE70000240500405405004005BD030067
:10AD4000C1AC030010B5202A04DB0146203A914033
:10AD5000002010BD914020239C1A0346E340194374
:10AD6000904010BD03460B439B0703D009E008C980
:10AD7000121F08C0042AFAD203E00B780370401CAB
:10AD8000491C521EF9D27047D2B201E00270401C39
:10AD9000491EFBD270470022F6E710B513460A465B
:10ADA00004461946FFF7F0FF204610BD30B50446B3
:10ADB0000020034600E05B1C934203D2E05CCD5CC4
:10ADC000401BF8D030BD0000064C0125064E05E0C2
:10ADD000E36807CC2B430C3C98471034B442F7D3BC
:10ADE000FFF772FF58F7030078F70300F0B500246F
:10ADF000151C1E1C8DB0139B029003911C571F1D28
:10AE00003B1C04A8111C0094029A00F0A4FC04A8A6
:10AE1000011C139A00F08FFC029804AA011C139BDA
:10AE200000F079FC281C291C04AA139B00F073FC79
:10AE30003B1C301C311C039A009400F08CFC04A8CD
:10AE4000311C139A00F077FC04A8011C029A3B1CE9
:10AE5000009400F080FC04A8011C2A1C3B1C0094F8
:10AE600000F079FC281C291C029A3B1C009400F07D
:10AE700072FC03982A1C011C139B00F04CFC1298D6
:10AE8000029904AA3B1C009400F065FC301C311CA4
:10AE9000129A139B00F03FFC301C311C039A3B1CA0
:10AEA000009400F058FC281C04A9221C00F0E3FCCC
:10AEB0000DB0F0BDF0B51C1C071C161C0D1C89B094
:10AEC0006846111C1A1C00F036FC381C391C6A46F6
:10AED000231C00F020FC68466946321C231C00F04D
:10AEE0001AFC281C291C6A46231C00F014FC09B01B
:10AEF000F0BD002A03D0013A8B5C8354F9E7704718
:10AF0000F7B51E1C01910223F15E051CC81DC31775
:10AF10001F315B0F1B18C817C00E41184911DB10F9
:10AF20000091141E9C4200D91C1C6B460027DF5761
:10AF3000281C391C00F068FA221C281C0199FFF714
:10AF4000D8FF0223F25EE400944220D9A41A002222
:10AF5000009B9B00EB18043B191D8D4209D2196818
:10AF6000081CE04002431A602022121B91400A1C78
:10AF7000F1E72436301C291C3A1C00F051FA012854
:10AF800005D0281C291C321C3B1C00F0D9FCF7BD45
:10AF9000F0B5002697B0049103939E57051C311C11
:10AFA000101C141C00F061FA002800D096E006A8DE
:10AFB0000499039A00F0BFFB039B0EA8291C06AA64
:10AFC00000F0A9FB06A8011C039A00F0B4FB04984A
:10AFD000039B011C221C00F09EFB201C211C039AD9
:10AFE00000F0A9FB039B281C1F1D291C221C3B1CD5
:10AFF000009600F0D9FA201C211C221C3B1C009654
:10B0000000F0D2FA201C291C221C3B1C009600F0E8
:10B01000A2FB281C291C221C039B00F07CFB201C8B
:10B02000291C2A1C3B1C009600F0BEFA281C3B1C65
:10B030000096291C221C00F0B7FA2B68281CDB079D
:10B0400013D53A1C331C291C00F0B2F9311C0590B1
:10B05000281C00F001FC224B059AF3189B00EB180A
:10B060001968D2070A431A6002E0311C00F0F4FBB1
:10B07000201C291C039A00F05EFB201C211C0EAA38
:10B080003B1C009600F067FB201C211C0EAA3B1CF9
:10B09000009600F060FB0EA8011C221C3B1C0096D1
:10B0A00000F059FB281C291C0EAA039B00F033FB5F
:10B0B00006A8021C3B1C291C009600F04CFB281C17
:10B0C000211C321C00F0D7FB201C0499321C00F01C
:10B0D000D2FB049806A9321C00F0CDFB17B0F0BDDE
:10B0E000FFFFFF3F00487047A8F60300F0B50025BA
:10B0F000EFB01C1C749B08901B7806910393749B03
:10B10000079202229B5E4EAF1F33DA17D20ED3187E
:10B110005B115BB20293013B9B000593059A26AB42
:10B1200056AED550D55195510122749B211C9A568B
:10B13000381CFFF7DEFE0122749B301C9A56A118C2
:10B14000FFF7D7FE0C246B461C57381C211C00F05F
:10B150008CF90390A84200D023E1301C211C00F0A0
:10B1600084F9039D0490002800D01AE1749B391CD7
:10B170002433181C029A039300F052F9049D01280D
:10B1800000D00EE10398311C029A00F049F9049DA9
:10B19000012800D005E1311C1EA8039A029B00F093
:10B1A0001CFA059B049A0EAE9A51301C0699079A18
:10B1B000749BFFF7A5FE029B301C311C00931EAA56
:10B1C000039B00F095FA029B5EAD391C009316A814
:10B1D000039B1EAA00F08CFA281C0899221C00F080
:10B1E0004AFBA3000593EB180793059A089B079861
:10B1F0009918221C00F03FFB749B36AF4433191C96
:10B20000381C221C099300F036FB211C749B103162
:10B210008900591804313EA8221C00F02CFB749BB5
:10B22000291C04331EA83A1C0094069300F093FADC
:10B23000749B2A1C0193381C3EA9079B0097FFF7BB
:10B24000D5FD1EA8011C069A231C00F0C6F9281C77
:10B250001EAA0799749BFFF72DFE049B301C0A93CE
:10B26000099B02990B93089B0D950C9300F0D2FA61
:10B270000299061C16A800F0CDFA051CB04200DAAF
:10B28000351CADB26F1E3FB2391C0EA800F086FB14
:10B29000061C391C701E864116A800F07FFB431E59
:10B2A0009841400006430AABB600F65826A8311C68
:10B2B000221C00F0E0FA059B2EA8F118221C00F0D9
:10B2C000DAFA1EA8211C00F09FF80123023D1E930C
:10B2D000ADB22FB2002F45DB749B1EAAA4331E68AB
:10B2E00026A8749B2EA9B047391C0EA800F056FB67
:10B2F000061C391C701E864116A800F04FFB431E29
:10B30000984140000643B6000AABF758002F27D0FB
:10B3100036AE301C391C221C00F0ADFA059B3EA84D
:10B32000F918221C00F0A7FA301C3EA91EAA749B33
:10B33000FFF7C0FD46A826A9321C069B009400F02A
:10B340000AFA749B301C01933EA926AA2EAB0096E4
:10B35000FFF74CFD1EA8011C46AA749B00F0DBF908
:10B36000013DB5E71EA8011C069A231C00F035F923
:10B3700026A82EA91EAA749BFFF79CFD039826A958
:10B38000029A00F04DF8012805D026A8011C039A66
:10B39000029B00F0D5FA26A84EA9221C00F053F813
:10B3A000051C281C6FB0F0BD00000000000000006C
:10B3B00070B50824E31ADB000133041C002003A548
:10B3C0005B1920C940CAAD1920C4184720C940CA1A
:10B3D000754120C420C940CA754120C420C940CA53
:10B3E000754120C420C940CA754120C420C940CA43
:10B3F000754120C420C940CA754120C420C940CA33
:10B40000754120C4404170BD002310B55AB28A4234
:10B4100005DA0024920001331450DBB2F6E710BDC8
:10B4200010B5013AD2B253B2002B07DB9B00C458CF
:10B43000CB589C4204D8F4D2FF2002E0002000E068
:10B44000012040B210BD002330B5013AD2B254B24F
:10B45000002C07DBA4000D590459013A6C4023432A
:10B46000D2B2F4E75842584130BD00231A1C10B53F
:10B470005CB28C4205DAA400245801332243DBB2CB
:10B48000F6E75042504110BDF0B51D1CA7B016ABF9
:10B4900003900591101C291C0493161C00F0BAF9A6
:10B4A000AB01181A83B200936B460027DF5F3D4B58
:10B4B000FC17E40EE4196411E4B23B4004D52027E4
:10B4C000013B7F423B43013364B29FB2211C06A87B
:10B4D000FFF79AFF3BB2A400002B11DD06AA141956
:10B4E0000022111CAF00BA4210D0B058984001435E
:10B4F000A1502021B058C91AC8400432011CF2E7FB
:10B5000006AB1819311C2A1C00F0B5F901246B0098
:10B510000193AF0006ABDB1902936B4600229B5EE2
:10B52000002B36DB0020031C019A41B2914216DA4F
:10B5300004AEA20092598900565806AA8A58B21A37
:10B54000D21AB24202D096429B415B420126361B80
:10B55000B60004AFBE5901307250C0B2E4E7E41A3D
:10B560006242624106AE301C291CD4B200F074F96C
:10B570006B1EAA009B0092599959D2070A43029860
:10B58000291C9A5100F068F90098013883B20093A1
:10B59000C3E704ABA4000398E1582A1C00F06BF940
:10B5A00027B0F0BD1F00008070B500251E1C04AB45
:10B5B0005D57041C2B1CFFF7FBFE002806D1301C36
:10B5C000211C2A1CFFF72CFF012805D0201C211C60
:10B5D000321C2B1C00F0B4F970BDF0B5061CA3B0F2
:10B5E0000F1C081C191C151C1C1CFFF73EFF002813
:10B5F00004D0301C211CFFF707FF77E002A8391C9C
:10B60000221C00F038F90AA8291C221C00F033F98A
:10B6100012A8211CFFF7F8FE01231AA8211C12937F
:10B62000FFF7F2FE02A80AA9221CFFF7F9FE002884
:10B6300057D0029B01930123019A1A4204D102A818
:10B64000211C00F009F927E00A9A01921A4204D15C
:10B650000AA8211C00F000F93DE000281EDD02A828
:10B660000AAA011C231C00F06BF902A8211C00F09F
:10B67000F3F812A81AA9221CFFF7D2FE002805DA57
:10B6800012A8011C2A1C231CFFF792FE12A8011C01
:10B690001AAA231C00F054F912A81DE00AA802AA55
:10B6A000011C231C00F04CF90AA8211C00F0D4F85E
:10B6B0001AA812A9221CFFF7B3FE002805DA1AA85F
:10B6C000011C2A1C231CFFF773FE1AA8011C12AAD6
:10B6D000231C00F035F91AA8291C221C00F042FA9C
:10B6E000A0E7301C12A9221C00F0C5F823B0F0BD61
:10B6F00070B50024061C1D1C90B014AB1C57684686
:10B70000231C00F03AF8301C69462A1C231CFFF762
:10B71000BBFE10B070BD30B51C1C0023051C91B0E1
:10B72000E3566846AC3400F028F82368281C6946C4
:10B73000984711B030BD30B5141C0022051C91B0E3
:10B74000A2566846AC3400F0A2F82368281C69466B
:10B75000984711B030BD70B500251E1C04AB5D5775
:10B76000041C2B1C00F0ECF8002805D0201C211C28
:10B77000321C2B1CFFF71CFE70BDF0B55F46564611
:10B780004D464446F0B4013B9B0098465B00994609
:10B79000002300240025002601B4002702E0370022
:10B7A00040463F1A9A46A346AC46B646F01B14588C
:10B7B000C859030C80B2250CA4B21E006E4363432B
:10B7C000454360431C041B0C00195E412C042D0CE6
:10B7D00000196E4153465C4665461B1874410020B3
:10B7E000454176460437474501DCB742DADD00982B
:10B7F000835123462C46002504364645CDDD4E4573
:10B80000CDDD835101BC3CBC90469946A246AB4677
:10B81000F0BD00000139C9B24BB2002B0ADA002397
:10B820000131C9B2994213D00A4A49B28A1892002A
:10B83000125804E09B001B58002BEBD0EFE7002AC6
:10B8400002D052080133FAE70139490159188BB285
:10B8500018B27047FFFFFF3F002210B58900411862
:10B8600004390B1D984205D20C68630813430B6022
:10B87000E207F5E710BD30B5002463B2934205DA64
:10B880009B00CD580134C550E4B2F6E730BDF0B5A9
:10B890005F4656464D464446F0B4013A9200904603
:10B8A00052009146002200230024002501B4002606
:10B8B00002E02E004046361A92469B46A446AE460B
:10B8C000AF1BCB598859020C80B21C0C9BB21500DF
:10B8D00065435A43444358431304120CC01855415E
:10B8E0002304240CC018654152465B466446BE42A0
:10B8F00003DA002712186B417C41002712186B41B4
:10B900007C4175460436AE4202DAAF1BBE42D3DD3F
:10B91000009842511A462346002404354545C6DDA9
:10B920004D45C6DD425101BC3CBC90469946A246FD
:10B93000AB46F0BD00000000000000000000000069
:10B9400070B50824E31ADB000133002403A5C046C8
:10B950005B1920C940CAAD1B20C0184720C940CA86
:10B96000B54120C020C940CAB54120C020C940CA45
:10B97000B54120C020C940CAB54120C020C940CA35
:10B98000B54120C020C940CAB54120C020C940CA25
:10B99000B54120C064416042604170BD1F234A111F
:10B9A00019401E3B8B409200105818407047000011
:10B9B000F0B50C1C00278BB00822051CFFF75BFFBD
:10B9C000E36A02A80593236B011C0693636B021CB8
:10B9D0000793A36B04970893E36B039709930823DA
:10B9E0000297FFF7E5FC291C061C02AA0823281C65
:10B9F000FFF7DEFC236B86190593636B02A80693A1
:10BA0000A36B011C0793E36B021C0893082309979F
:10BA1000FFF7CEFC291C361802AA0823281CFFF7C2
:10BA2000C7FC236A36180293636A291C0393A36A2E
:10BA300002AA0493A36B281C0893E36B079709934E
:10BA4000082306970597FFF7B3FC636AA26B02937E
:10BA5000A36A06920393E36AE26B0493636B36185E
:10BA600005930893236A07920993291C02AA0823C5
:10BA7000281CFFF79DFCE36A36180293236B291CF0
:10BA80000393636B02AA0493236A281C0893A36A96
:10BA900007970993082306970597FFF751FF236B34
:10BAA000361A0293636B291C0393A36B02AA0493B7
:10BAB000E36B281C0593636A07970893E36A06976C
:10BAC00009930823FFF73CFF636B361A0293A36BBD
:10BAD000291C0393E36B02AA0493236A281C059391
:10BAE000636A08970693A36A0793236B0993082355
:10BAF000FFF726FFA36B361A0293E36B281C039310
:10BB0000636A291C0593A36A02AA0693E36A049751
:10BB10000793636B0897019309930823FFF710FFBE
:10BB2000341A0F4EBC4216DA321D281C291C082379
:10BB3000FFF73EFC0419F7D410E0301D291C082241
:10BB4000FFF76EFC012809D0321D281C291C082390
:10BB5000FFF7F6FE241A002CEFD0F5E70BB0F0BD8E
:10BB6000A8F6030070B5141C0268051C0B1C002607
:10BB7000D20705D51A1C291C231CFFF719FC061C2B
:10BB8000281C211CFFF768FE002E08D0044BE41887
:10BB90008023A400281902681B061343036070BDAC
:10BBA000FFFFFF3FF0B5141C8DB0051C0E1C04A850
:10BBB00000212022FFF7F1F803232778281C311CED
:10BBC000221C7FB20493FFF7B6FD231D281C291CFD
:10BBD00004AA00970393FFF7BEFD281C291C321C02
:10BBE000231CFFF798FD221C00978432281C291C77
:10BBF000039BFFF7D9FC0DB0F0BD00008307FF22C7
:10BC0000DB0E9A408907090E994000280BDA0007DD
:10BC1000000F0838830808489B001818C36993432D
:10BC20000B43C3617047830804489B001B181868C6
:10BC3000904308431860704700ED00E000E400E026
:10BC4000BFF34F8F04490348C860BFF34F8F00BF55
:10BC5000FDE700000400FA0500ED00E01CB500243B
:10BC60006846047000F06EFA03F04EFA002818D10E
:10BC70000E480168002914D00D498968C907C90F09
:10BC80000FD004600B4880686946087101A90A4812
:10BC900002F09CF8084802F083F8002801D002F076
:10BCA0000FF86846007800F06BFA1CBD00D1004028
:10BCB00000D3004000D5004070F5030010B50649E0
:10BCC0000020086048608860C86003494039086007
:10BCD000486003F0B7FA10BD4011014010B503F001
:10BCE00023FA10BD10B506484068002805D08047EB
:10BCF000002801D000F0E0F810BD01F057F810BDA9
:10BD00007026002010B501F0A1F8002805D01F49C9
:10BD10001D484860C8131E4988611E48018CC9B27D
:10BD200001290BD1828C120708D1028D1206120F45
:10BD3000042A03D1828D1206120F0AD0012921D1C3
:10BD4000818C09071ED1018D0906090F0A2904D02B
:10BD500007E0114A01219160F5E7828D1206120F6A
:10BD600005D00D290ED1808D0006000F0AD10B4899
:10BD70000168012904D00A49016001680129FCD148
:10BD8000C021416110BD0000DFFF07C00005004079
:10BD9000006C0040C00F00F00006004000EC0640C0
:10BDA0007593000030B47446641E2578641CAB4261
:10BDB00000D21D46635D5B00E31830BC184702E00B
:10BDC00008C8121F08C1002AFAD170477047002026
:10BDD00001E001C1121F002AFBD17047202804DABC
:10BDE000012181400348014201D001207047002019
:10BDF00070470000FC06FFBC86B00B2269468A82B1
:10BE000002220A7001234B7088700320C8700A71E7
:10BE100059204871FE20887102A805A901307DDFF4
:10BE2000002816D16846808A0B2807D8411C6A462C
:10BE3000D17109210930117280B205E00C206946E8
:10BE4000C871082008721420C1B200231A4668463F
:10BE500072DF06B07047000010B5144C86B0207A2F
:10BE6000800702D5002006B010BD18216846FEF7F5
:10BE700092FF0620FFF7C0FF0028F4D16946087042
:10BE80000190087228220A824882684673DF0028DF
:10BE9000E9D1012006494005C860162001F038FFAD
:10BEA000A06802210843A060DCE7000018260020FB
:10BEB00000050050FFF7C4FEFFF7C2FEF7B5244CA3
:10BEC00082B060880E4681423FD800256846214FE7
:10BED000057000F037F922786078A188884201DA8D
:10BEE000401C00E00020C0B2904204D168460078B7
:10BEF00000F046F927E065786078884201DA401C56
:10BF000000E0002060706846007800F039F9BD421A
:10BF100019D0A068EF000499C151029900290CD0F2
:10BF2000002E0AD0608832464543E0682818FEF7A4
:10BF300019FFA0683818868002E000213818818037
:10BF4000002005B0F0BD0420FBE70920F9E7000060
:10BF500030260020FFFF000010B50D4C03E0401C10
:10BF600000E0002020702078617881420FD0217895
:10BF70006088E26848438018A368CA00D1189A58BC
:10BF8000898890472078A1888842EADAE7E710BDDF
:10BF90003026002030B5CB0008339DB29307002433
:10BFA000002B01D0072030BD044B9A605219DA6093
:10BFB0005C701C7058809980002030BD30260020B5
:10BFC0000A4B5B68002B07D0002A07D0002805D059
:10BFD0000068037C002B03D00820704707207047BF
:10BFE00000230374417442611846704750260020B4
:10BFF00010B50446082902D00020FFF75DFF216834
:10C000006068884710BD00001CB501910090034A8C
:10C0100008216846FFF752FF1CBD0000F1BF030076
:10C02000FFB507469007002581B01E46144600283C
:10C0300025D1002C23D002F0D3FD3046114EF06004
:10C04000304610300570457002998170446075600B
:10C05000357001240C4875702405046003211420F8
:10C06000FFF7CCFD09480460094CA76003211120AB
:10C07000FFF7C4FD6068B060002005B0F0BD072088
:10C08000FBE700004026002080E200E000E100E045
:10C0900000150140FEB51F4B5B68002B30D0002817
:10C0A0002ED0052901D20720FEBD4369002B27D0E1
:10C0B000437C012B26D000270291044600256946C7
:10C0C00016460D70684600F03DF801A803F036F9F9
:10C0D000002819D0012101700F494460496881602E
:10C0E000029907614661C16068460A490079487053
:10C0F0006846007800F044F803F058F82846FEBD82
:10C100000820FEBD0F46D7E768460425007800F0FA
:10C1100037F8F3E7502600200015014010B5084914
:10C12000496800290AD0002808D04169002905D0B3
:10C1300000210174022103F061F810BD082010BD38
:10C140005026002030B5EFF3108172B6094A5468CA
:10C150000123002C04D00370002900D162B630BD49
:10C160005360054B1D68054C254015601C6000227E
:10C170000270F1E76426002080E100E0FC06FFBCCD
:10C1800008494A68002A0CD000280AD1EFF3108031
:10C1900072B60A68044B1A6000224A60002800D177
:10C1A00062B670476426002000E100E070B50546E5
:10C1B00001461C220E48FEF7D5FD0E4C00262670C7
:10C1C0002968002906D00822201DFEF7CBFD201D7E
:10C1D0007ADF02E00748001D7BDF002807D1401E00
:10C1E00060806670044A00210448FFF7E9FE70BDD4
:10C1F000542C002004260020D9F2030004F503008B
:10C20000F8B5214C0146028800261E48E589102A0F
:10C2100013D01E4F112A1FD0122A2BD0502A1AD108
:10C22000881DC988A94216D14189022913D10C3031
:10C2300000F016F900280CD112E08A8804464280EA
:10C24000104808220C301831FEF78CFD6670002D66
:10C2500001D100F0B5F9F8BD0021C9434180467015
:10C260003868FFF75BFF0028F5D0A1690029F2D0FC
:10C270008847F8BD034808220C300831FEF772FDEC
:10C28000E7E7000004260020542C002004F50300FA
:10C2900010B502480068FFF741FF10BD04F5030028
:10C2A00070B505460020C043134C86B0208001269F
:10C2B00068468674114901822A4604A93046A0DFE7
:10C2C000002817D10E4B0FCB03936B4607C3A91C55
:10C2D000684663DF00280DD1284600F0CDFB00281A
:10C2E00008D1284600F096FA002803D1A068304310
:10C2F000A060002006B070BD1826002059FE000086
:10C300000CF5030070B51A4D0024A868410701D54B
:10C31000002070BD04210843174AA8601549174B37
:10C32000126800BF00BF00BF00BF00BF00BF00BF5A
:10C3300000BF9A4200D000BF0139F2D12A881049CB
:10C340008A4205D01321104676DF0400E1D10BE0CC
:10C35000800709D574DF0400DBD1152001F0D8FC7B
:10C36000A86802210843A860FFF792FF204670BD2D
:10C3700018260020C0D40100842600200024F400E8
:10C38000FFFF000000B587B0152001F0B7FC1620B4
:10C3900001F0B4FC152001F0BBFC162001F0B8FC44
:10C3A00024480068059001F0E1FA002817D12248DE
:10C3B00013DF002813D1214B4822214905A802F0A0
:10C3C00077FE002801D0FFF777FD01216A46084675
:10C3D00002F042FE002802D1684602F033FE002837
:10C3E00026D1184802F024FE002821D100F0AEFC2E
:10C3F00000281DD112484830FFF752FF002817D1FE
:10C400001C216846FEF7C7FC0F48019001208003FD
:10C4100002900320694608730020C88108740B4805
:10C4200006906846FFF7C2FE002801D1FFF714FD11
:10C4300007B000BD08F5030000AC030095F0030051
:10C44000702C002051C40300CD0C0000B9C50300BE
:10C4500010B50446FFF7D4FE204601F00FFD10BDD5
:10C460004178027808021043C007C00F70470000EF
:10C4700010B50349085C012101F052FC10BD000019
:10C48000FCF4030010B50349085C002101F048FCEE
:10C4900010BD0000FCF403007CB50024074E2546C7
:10C4A000305D0122009500231146019501F012FC38
:10C4B000641C042CF4D300F003F87CBDFCF40300EE
:10C4C00010B500242046FFF7D3FF641C042CF9D3D9
:10C4D00010BD10B543689C184460002904D105E0E4
:10C4E00018780870491C5B1C521EF9D2012010BD3F
:10C4F000002807D00449814204D80449814201D967
:10C5000001207047002070478826002098260020D0
:10C51000F8B52348416800293ED00E6821494C688F
:10C5200087688078E11B0D022D0AED1C002814D1CC
:10C5300001201D4A000450601B4A403A50601B49CC
:10C54000400008601A4908601A49012008602F203D
:10C5500000F0DEFD124901208870B54200D2354658
:10C56000E81900020F4B000A403318600D4A516869
:10C57000001B091B0902090A0002000AC91C8142AA
:10C5800009D9506818602F2000F0C2FD012007492A
:10C59000400480390860F8BD02F022FBF8BD0000BD
:10C5A00040260020001501404013014080E200E0D9
:10C5B00000E100E00010014010B5FFF77DFC10BD68
:10C5C000F8B5164800F034FC144D00260C3D144C10
:10C5D000002807D0616900291CD001206A4610702C
:10C5E000684616E02878002805D06169002911D036
:10C5F000684606700DE0687800280DD0A1680948EB
:10C6000000220068FFF746FD002803D0A169002939
:10C6100000D088472E70F8BD6168F0E71026002032
:10C62000542C002004F50300F0B50026F643002A40
:10C6300004D01268D2430023094F0DE03246FAE7D6
:10C64000C45C624008245508D20700D032463A4004
:10C650006A40641EF7D15B1C8B42F1D3D043F0BD1E
:10C660002083B8EDF0B5146907462068251D8DB00C
:10C670001646002819D002291BD00A2000906B46CC
:10C6800009AA384602F007FA00280CD009A901A827
:10C69000009A02F0DDF801AF0FCF0FC72368716871
:10C6A0002A4605A898470DB0F0BD384602F044F977
:10C6B000F9E76946384602F0D3F80028F3D023683A
:10C6C00071682A46684698470028ECD002980028EE
:10C6D000F5D1019878600120E5E710B553685B78E3
:10C6E0009B099B0103D0402B04D0002010BD00F01B
:10C6F00005F810BDFFF7B6FF10BD0000F0B50F46FE
:10C7000051680646487814460207120F324D9300CE
:10C71000ED58302385B0184006D0102806D02028C8
:10C7200008D0302855D140E022694FE061690120EE
:10C73000087049E0022F2AD1042A28D8012000904D
:10C7400001A93046676902F08BF800281DD00AE085
:10C750000A7942432069121801A8A847002810D07E
:10C760003878401C38700398002804D06168387805
:10C770004A799042ECD3029870600398002828D13F
:10C7800002E000200090F6E7009805B0F0BD626975
:10C790000B791078276943434979DB19884218D20D
:10C7A000401C10701A46616810E008786169072A19
:10C7B000087009D1606801792069FEF7ECFA6068B9
:10C7C0002169806802F067F8226961683046A847ED
:10C7D000DBE70020D9E7000084F6030010B50B4921
:10C7E00009480B4A096800BF00BF00BF00BF00BF77
:10C7F00000BF00BF00BF914200D000BF0138F2D19E
:10C80000FFF7AAFB10BD0000A086010084260020CF
:10C810000024F40030B58FB004461C216846FEF7B2
:10C82000BAFA142109A8FEF7B6FA00206946079063
:10C830000A7808210A4310231A4369460A70A2782D
:10C8400008A98A700125694602070D84120F0A772C
:10C85000EA184A778A7FF9210A40921C1A432A4330
:10C8600069468A7708A9099107A917220A9169469A
:10C870000A860D90234620880C3309AAA2DF0FB048
:10C8800030BD000002488168491E81607047000089
:10C89000E02500201FB50E480146826B5C316846DA
:10C8A00001F0D6FF6C460ECC0A480EC009490A4872
:10C8B000C8600A49002008604860094A09490548DB
:10C8C00001F05EFD002800D0012004B010BD000082
:10C8D00000300020242C0020C1E60300FC250020AD
:10C8E0009826002090F40300F8B50646041D0020A9
:10C8F0009C461146002A2BD01A0029D05F22125DD7
:10C90000002A03D06022125D012A21D0227A002A57
:10C910001ED0E268332A1BD10022257C16E00327B3
:10C9200093003F031B19BF895B69BFB2BB420CD1A7
:10C93000254620356B794B4A002B0BD0012B12D0AA
:10C94000022B0CD0032B03D109E0521C9542E6DCEC
:10C950000A20F8BD20780028FAD0906803E02078FB
:10C960000028F5D0D068002B04D0022B06D0032B72
:10C9700007D103E062688242EAD302E06268824241
:10C98000E6D937466037387C0028E1D13748364A47
:10C9900002602022426003466246052000F07CFBD4
:10C9A0000028D5D1304831467A7C72312030FEF7EC
:10C9B000D9F92E482C49083820310160797C416032
:10C9C00003462A4A2A49042000F08CFB002801D0A3
:10C9D0000520F8BD254E00201C3E30616A79002AF2
:10C9E0002BD0012A34D02348FF218902081A022AB9
:10C9F00028D0032AACD1297B0029A9D0A979002904
:10CA0000A6D0A26A216B53183361002A26D00029D0
:10CA100024D081420FD8214620223F311248FEF710
:10CA2000A1F93069002819D0104A0021103A00F00D
:10CA30004BFE002814D00420F8BD287D002887D0A4
:10CA4000A06B09E0297B002982D0216B3161E0E7EE
:10CA5000A879002885D0A06A3061DCE70320F8BD02
:10CA60000120F8BD00300020C42B0020FC25002050
:10CA7000F4F4030000AC030010B58EB004461C2192
:10CA80006846FEF788F9142109A8FEF784F9002208
:10CA90006946079208780421084369460870A0781F
:10CAA00008A98870022069460884501C0007000FFE
:10CAB0000A7710304877887FF92108400121801CCF
:10CAC00008436946887708A8099007A80A901420A7
:10CAD00008860D922088231D09AAA2DF0EB010BD82
:10CAE000044A002901D1002313705268002A00D0A3
:10CAF0001047704728260020F8B51C4617460D46FB
:10CB000006001ED0002D1CD0002C1AD000F0C2F957
:10CB1000002818D0284600F0BDF9002813D0204680
:10CB200000F0B8F900280ED0FEF7DCFA009023469A
:10CB30003A4629463046FEF7D9FA002805D00020AB
:10CB4000F8BD0E20F8BD1020F8BD0B20F8BD000088
:10CB500010B50E4900230A784C78A24212D0521C1C
:10CB6000D2B20A70022A00D10B700A78074B9200E9
:10CB700018339A580260886810180002000A88600A
:10CB8000012010BD0360002010BD000040260020E1
:10CB9000F8B506461C481F46007815460C46C007E7
:10CBA0000AD03046FFF7A4FC002807D0002C07D09D
:10CBB000A00507D00620F8BD0120F8BD0220F8BD71
:10CBC0000320F8BD3068A04204D8A802716800199B
:10CBD000884201D90520F8BD002D10D0684601F02B
:10CBE000EFFE00280DD000980221C0C00170A10105
:10CBF000090C8180058101F035FF0020F8BD04207B
:10CC0000F8BD0720F8BD00006C26002030B4094BA9
:10CC100002241A68520852001A60002906D02243E2
:10CC20001A604268002A03D030BC1047A243F7E7DD
:10CC300030BC7047242600200348012201781143AC
:10CC400001700020704700006C2600200348406EF1
:10CC5000042801D000207047012070478C3100204B
:10CC6000F8B507461E481E46007815460C46C00714
:10CC70000ED03846FFF73CFC00280BD0002D0BD01F
:10CC8000002C09D028462043800707D00620F8BD95
:10CC90000120F8BD0220F8BD0320F8BD3868A0428D
:10CCA00004D8B10078680919884201D20520F8BD7E
:10CCB000002E11D0684601F083FE00280ED00098A7
:10CCC00006990760416001210172C5600461868296
:10CCD00001F0C8FE0020F8BD0420F8BD0720F8BD13
:10CCE0006C26002070B5174B0446186E1821484377
:10CCF0001549C0180A78950715D5022C02D0032CC7
:10CD00001CD102E001F0B4F918E04A78521CD2B20A
:10CD10004A70032A12D900224A70082101F0C4FF88
:10CD200001F038FE0AE0500708D5FB2002400A70E7
:10CD3000586E002802D0022002430A7001F05CFE07
:10CD400070BD00008C3100206C26002010B500243E
:10CD500086B0601C0007000F0194694610300294F1
:10CD6000087003A871DF002819D16946487B401C70
:10CD7000487303A9002070DF002810D1072209A101
:10CD800068467CDF00280AD10C2168468180182182
:10CD9000C180FF2104819131418101A87ADF06B071
:10CDA00010BD00004466755461726700F8B51F4CF1
:10CDB0002078002839D02069002807D00026E068B4
:10CDC000002805D00025002E04D014E00126F6E747
:10CDD0000125F8E76078002827D1684652DF05284A
:10CDE00004D0002804D0FFF767F804E0012602E031
:10CDF000216900988847002D13D16078002814D14C
:10CE0000608869460880A06861DF052804D0002892
:10CE100004D0FFF751F804E0012502E0E168A068C2
:10CE20008847002ED6D0002DCDD0F8BD702600202A
:10CE3000418805480288914204D34088814201D844
:10CE40000120704700207047082600201048018C00
:10CE5000C9B2012917D1818C090714D1018D0906A6
:10CE60000A0F03D1828D1206120F0ED0090F01296D
:10CE700003D1828D1206120F07D0032903D1808DB2
:10CE80000006000F01D0002070470120704700000D
:10CE9000C00F00F0800701D00020704701207047CC
:10CEA00070B5054608680C4686684A6831462846CB
:10CEB00001F018FC6068286120460C3068617078C9
:10CEC0008009022801D1241D2C6170BDF0B5284CC9
:10CED0002146103948688B68227886469C46CF7870
:10CEE000667836E0182353436168521CC918A3784A
:10CEF000D2B2934200D100220B78022B02D0032B36
:10CF000027D123E003464D68194603E0A94204D027
:10CF10000B46C96900291CD0F8E7002919D08B42BB
:10CF200008D1C069002805D1124F0125BD60002538
:10CF3000AC4601270D68C969D961002909D00B6881
:10CF40005B190B6005E00174C06900E00021002856
:10CF5000F9D19642C6D10649624610398A604860C6
:10CF6000CF70704501D00120F0BD0020F0BD000061
:10CF70005026002000100140F8B52C4E0446706881
:10CF80000025009041E0002C02D02046E46920E01A
:10CF9000264818231030017842684B43491CC9B217
:10CFA000D21801708378994200D1057011785068C9
:10CFB00001292CD1017C002929D191684160D168D7
:10CFC00081601169C16051698161F178002900D0E7
:10CFD00045604368B268164F991A0902090AB942B6
:10CFE00002D28268891806E0D11A09028268090A09
:10CFF0008A4202D9511A016000E0056045600121B2
:10D0000085600174C56102F0D9F8002CBBD10748D6
:10D010001030017840788142BAD17168009881421D
:10D0200001D00120F8BD0020F8BD000040260020FE
:10D03000FFFF7F0010B5FFF72FFA0220FFF722FA5B
:10D0400008490748086000F023F8002801D0FEF7DF
:10D05000F7FD03200003806800F006F8002010BDF3
:10D060000C0003005007005010B5044600F07EFC91
:10D07000002809D10549401E0860204613DF00281A
:10D0800002D12046FDF728FE10BD000080E100E03F
:10D0900010B500F0EDFB10BD70B59CB01C461546F8
:10D0A0000E46052802D006201CB070BD60682028FE
:10D0B00001D00920F8E7684601F0B6FE0028F3D158
:10D0C0002A463146684601F08BFF0028ECD1012248
:10D0D0006846216801F020FE0028E5D1202060602C
:10D0E0000020E1E770B5042801D0062070BD486833
:10D0F000402802D15868402801D0092070BD30CAAC
:10D1000008681B682A462146FFF7F6FC70BD000040
:10D1100000280FD00849094A096800BF00BF00BFB6
:10D1200000BF00BF00BF00BF00BF914200D000BFE2
:10D130000138F2D170470000842600200024F4005A
:10D14000F1B50320274D00038268286B6E6A121820
:10D1500082B0371A00920124A402A74200D83C46AC
:10D1600000220121009800F0E9FA002838D10023BC
:10D1700022460299009800F043FB002830D1224655
:10D180000299009800F0C6FB002829D10022012155
:10D19000029800F0D3FA002822D1286B00192863E6
:10D1A000002000F023FD009800190090029800195B
:10D1B00002903F1BCFD1032000038068002231463C
:10D1C000FFF732FAA96A814203D10121AE612962D7
:10D1D000E8610448243000F091FB002000F006FDD7
:10D1E000FEBD00000030002010B50A4C206A012866
:10D1F0000CD1E06900280BD003200003A1698068EE
:10D200000022FFF711FAE169814201D0002010BD30
:10D21000012010BD0030002070B50D460A680B4992
:10D22000496B541A0E1822463146094800F072FB29
:10D23000002804D02146304600F07AFB70BD284615
:10D2400000F05CFB002000F0D1FC70BD003000203D
:10D2500000AC0300F8B51446404F0A780E4601258D
:10D26000B96BF86B1300FEF79DFD077605203B1C9C
:10D27000766E7600B068002805D0FF210131884223
:10D2800003D90420F8BD0320F8BD3548002484707C
:10D29000324820213830FDF77EFD3C63B068B8632A
:10D2A0005AE06060386CA06056E0B26813188B4298
:10D2B00003D96060386CA060E5E7284B71685C3387
:10D2C000C018FDF74FFDF86BB168244A4018F863A9
:10D2D0004032B1687068FFF7A7F93864F86BE0E78F
:10D2E000884201D00820F8BD1D4CA078002801D04C
:10D2F0000120F8BDFFF7CEFA012822D11948007DA0
:10D300000028194818D0783082781849012A01D0AD
:10D3100005200CE0124A1C320CCAFFF7E5FA01287E
:10D3200005D1002000F062FC002802D00A2005464A
:10D3300012E00120A0700FE00078002801D00A253B
:10D340000AE00520F8BD386CA060F86B6060FF2033
:10D350000130206000E002252846F8BD00300020A2
:10D36000E0250020F826002098260020242C00200C
:10D3700010B5024603200A4B0003816818461C6959
:10D380001830012C08D05C69002C05D09B69054C35
:10D390000C301B19A343591800F006F810BD00000B
:10D3A00000300020FF030000F8B50D461646014688
:10D3B0008A680020012A0DD00127A52A12D0AA2AA6
:10D3C0001ED0AC2A0DD10C46284600F0A3FB002845
:10D3D00014D119E00F494969012902D12846FFF704
:10D3E000AFFEF8BD28460C4600F094FB002805D19E
:10D3F000204600F083FA002000F0F8FB3760F8BD0B
:10D400002846FFF709FFF8BD21462846FFF704FF2D
:10D41000F4E7000000300020FEB50120009097489E
:10D420000E788078964F019015460C46BA6C396D8F
:10D43000786D3300FEF7B6FC07F2053AF7F3F2EF2A
:10D44000F200A168002946D08C4A8B05126902D0EF
:10D45000431893423FD101231B03994232D8019BC9
:10D46000864D002B7ED0411891427BD8F96CB9646F
:10D47000A1683865796438636978824A491C8907EC
:10D48000890F69700021A980A968491CA960A16859
:10D490008918EA68890A80187B4A00F04FF9002849
:10D4A0007ED0A868401EA8600520FEBD6960B86CEB
:10D4B000A8600198714E0028D4D0FF20A1680130E7
:10D4C000814201D90420FEBD386D7A6D0818801A9A
:10D4D0007A6C904201D90320FEBD694A60684832E7
:10D4E000FFF7A2F866498864086DA268801808658D
:10D4F0006860886CA860B088A2681118FF2907D8F6
:10D50000717867680B02614959180818394643E079
:10D51000FF210131091A8FB2717863680A025B49F1
:10D52000511808183A461946FDF71CFCB088C01976
:10D5300082B2B280A068D21CC01BA0606068920852
:10D54000C0194F4F6060386BF1684018B168491CD2
:10D55000B16071780B024D4959184B4B00F050F9EE
:10D56000002800E063E04CD0B068401EB060F86C6A
:10D57000B864786D38656860F86CA86070780021D0
:10D58000401C8007800F7070B180A268002A71D0A3
:10D5900003023E4861681818FDF7E4FB208900E0AB
:10D5A0002EE0B18840180104B080090C62D0344CE0
:10D5B000626D206B636C821A52189A425AD3F268D9
:10D5C000C91C8018B268521CB2608A0871780B02BC
:10D5D0002E4959182C4B00F013F9002816D0B068CA
:10D5E000401EB060E06CA064606D20656860E06C17
:10D5F000A8607078401C8007800F70700020B08099
:10D6000038E0B188386B40183863B7E7B188206BD1
:10D6100040182063EDE727E001E004E02CE06960BA
:10D62000B86CA86026E07B6C081A984201D00820EC
:10D63000FEBDFA6400207965786400F0D7FA00280E
:10D6400001D00A20FEBD0D4C386D2169884202D000
:10D6500010E000F031FBA0680028FAD10B48B03888
:10D6600000F090F9009005E0AA60386D6860012034
:10D67000000328600098FEBD0220F3E7E0250020AB
:10D6800000300020FF03000085C80300C4270020ED
:10D6900010B50B480069000DC007C00F0ED0094837
:10D6A000816D012901D0002010BD0021816508464F
:10D6B00000F09CFA002801D0FEF7FEFB012010BD0F
:10D6C0000005005000300020F0B58C4618490324B6
:10D6D0004B69032109038968A4025B1A1F1B874257
:10D6E00015D3144C11602346183B196A00250129F3
:10D6F00001D01D610EE0104E216889198E0AB60214
:10D70000BF1B0121B84207D96246002A01D004207C
:10D71000F0BD19615D6106E01D61064C596111683B
:10D720000C34711811606560A56020600020F0BDA8
:10D730000010001018300020FF030000F0B50E4666
:10D740002049044608681546002785B0420719D5C8
:10D75000820702D50A2005B0F0BD01221949104305
:10D760000860B2B22B4621461748FFF711FA0700AE
:10D770001448016802D04908490001E00122114320
:10D7800001601DE0A001000C0490204600F0D4FAD6
:10D79000012080022418761EF7D1002D10D00B4AEC
:10D7A00091681068D26802910090019503926946D1
:10D7B00004980881A001000C488100216846A84710
:10D7C0003846C8E724260020882600201CF50300E0
:10D7D00010B501460020084C00290BD0FFF72CFAA9
:10D7E000002804D1054801F095FC002801D008204C
:10D7F00010BD0421216010BD24260020E5CC0300CB
:10D80000F0B51646184A074610681C46002585B034
:10D81000430717D5830702D50A2005B0F0BD0123C1
:10D82000114A184310600A46B3B239460F480094B3
:10D83000FFF716FA0500F0D10B48012201681143E9
:10D8400001600EE03246384600F08CFA002C08D019
:10D850000020009003900297019468468681002181
:10D86000A0472846D9E7000024260020882600206B
:10D8700038B50020009000F091F96846FFF778FD78
:10D880000124002800D00094FFF702FF002801D0F7
:10D89000009411E0009800280ED1FFF7A5FC0028A5
:10D8A0000AD0FFF7A1FC002804D003200003806801
:10D8B000FFF7DAFB002038BD0E4B0F4A0521002090
:10D8C000FEF7AEFB002801D0FEF7F6FA0A4A142153
:10D8D00078320820FEF75EFB002801D0FEF7ECFA54
:10D8E00000F0D4F90028E6D100F0C8F8FEF734FBC8
:10D8F000FCE7000009C00300DC2C002000210160CF
:10D900004160816002480163416301614161704788
:10D91000003000201FB5054B92081B6A01AC009334
:10D9200007C4684618DF04B010BD00002CF50300E2
:10D930001FB58908002201AB009207C3684618DFB3
:10D9400004B010BD1FB5920813061B0E02D00920AB
:10D9500004B010BD044B1B68029000930392019128
:10D96000684618DFF4E700002CF503001FB5044BF0
:10D970006C460FCB0FC4684618DF04B010BD000022
:10D980003CF50300F8B5074604462037787F0125AB
:10D99000032808D00A25354E706900281DD00128BB
:10D9A0001ED00A20F8BD334E314830602020334667
:10D9B000706018461C380269C1680520FFF76CFBCF
:10D9C000002800D00A25214620223F313068FDF78B
:10D9D000EDF90028DFD00525DDE72448183001E007
:10D9E00022482430012D03D000218160416027E0CE
:10D9F000797900290ED001290ED002290ED00329F1
:10DA00000FD00A257979002910D0022911D00329D5
:10DA100011D10EE0012102E0A52103E0AA218160DD
:10DA2000F0E7AC218160A16A7163EBE76168B160E6
:10DA300001E06168F160B16C41600E491C3909690F
:10DA400001600A4820213830FDF7A5F90748FF2278
:10DA5000B2215C30FDF798F900203063064800F0F1
:10DA6000C5F8002800D00A252846F8BD003000205F
:10DA7000C42B0020FC25002051E0030070B50120DC
:10DA8000FFF7A6FE002821D1114D124CA860A06B13
:10DA900000281AD0FEF7FEFE002816D0206A0028C3
:10DAA0000BD1A069002808D0094A00210C32286156
:10DAB000FFF70AFE0120A87007E0E06A002804D101
:10DAC000A069002801D0606AEEE7002070BD000068
:10DAD000E02500200030002010B50C780C4B012C04
:10DAE00001D0062C07D10C79012C03D0022C01D0D7
:10DAF000072010BD1C701B78012B03D0022B04D013
:10DB0000052010BDFFF7A6FB10BDFFF785FC10BD7B
:10DB1000E0250020F8B5034619480122016B1203E5
:10DB20008E18426B174D541A6419AC43A7087D191F
:10DB3000AD0AAD02CF18002A03D0914201D10020D6
:10DB4000F8BD2A4639463046FFF7FCFE0028F7D1DB
:10DB50002A4639463046FFF7DDFE0028F0D1761917
:10DB60007F19A54201D9002400E0641B0448416BE1
:10DB7000091B0163002000F039F8002CE1D1F8BD49
:10DB800000300020FF03000010B500225821024899
:10DB9000FEF74AFD10BD00000430002070B51049AA
:10DBA00000200870FF255D352A460E490E48FDF716
:10DBB000D9F80D4C2068401C04D0FFF7E5FF216820
:10DBC00081420CD029460848FDF7E5F80120606045
:10DBD000002000F00BF8002801D0FEF76DF970BDB1
:10DBE0002826002000FC03000030002070B5054608
:10DBF000164C01E0FEF7F2FD20780028FAD1012052
:10DC00002070656001F0B0FB002201211048FFF791
:10DC100095FD0728F6D00025002814D1FFF7B4FFA2
:10DC20000C49FF225D320860881AFDF79BF801F06D
:10DC30009BFB094B572209490548FFF7E1FD0728DF
:10DC4000F5D0002801D02570032070BD28260020C3
:10DC500000FC030000300020E1CA0300A42E0020D5
:10DC600070B50848084D401BC6080020044606E071
:10DC7000E000401940688047002802D1641CB4428B
:10DC8000F6D370BD80F7030078F7030070B508483D
:10DC9000084D401BC6080020044606E0E00040197D
:10DCA00000688047002802D1641CB442F6D370BDDE
:10DCB00080F7030078F7030010B5FEF74DF910BDAB
:10DCC00002490120886002490860704700D3004083
:10DCD00004D0004070B552000A439900049D0A43E5
:10DCE0002902059E0A43310405240A4324078000C3
:10DCF0000721001909024018026070BD05221207B1
:10DD000080008018072203211202801801607047EA
:10DD100001218140014881607047000000050050EA
:10DD2000012282400348002901D082607047C2600E
:10DD30007047000000050050084A02215160084960
:10DD40000B68002BFCD0906008680028FCD00020F5
:10DD5000506008680028FCD07047000000E50140D2
:10DD600000E40140F0B50C4D01236B600B4C2368BF
:10DD7000002BFCD0002306E09E008F5987512668B7
:10DD8000002EFCD05B1C9342F6D300206860206814
:10DD90000028FCD0F0BD000000E5014000E4014097
:10DDA000016880684A68824201D2521C00E0002269
:10DDB0000868824201D101207047002070478068C6
:10DDC000884201D9481C704700207047FEB50446C0
:10DDD0000E4600206946019008706846FEF7B2F9C9
:10DDE0002046FFF7DDFF07000AD0207C002807D07F
:10DDF0000420019068460078FEF7C2F90198FEBD44
:10DE00002068416820460D46FFF7D9FF2168002FA2
:10DE1000486006D0206801682046FFF7D0FF2168DF
:10DE20000860E268012A15D0022A17D0042A1AD005
:10DE3000082A1DD010466168684308183146FCF76F
:10DE400091FF204600F01CFE21688A688242D1D2F0
:10DE50008860CFE7616830784855F2E761683088BC
:10DE60006A008852EDE761683068AA008850E8E7E8
:10DE7000626803CEEB00D21803C2E2E770B5044635
:10DE8000314D00882E8814284CD00DDC022836D065
:10DE900010281CD0112828D0132817D100231A4687
:10DEA000852130467FDF0DE0502847D051282AD009
:10DEB00052283DD0552809D1A079002806D1132138
:10DEC000304676DF002801D0FDF7F6FF70BD012057
:10DED0001E498005C8601520FFF71AFFA08828801A
:10DEE000A86802218843A86070BDFDF7B5FF00282F
:10DEF00001D0FDF7E1FF0020C043288070BD002164
:10DF0000304667DFDEE7A0790028F7D021461048C9
:10DF100000F0D8F80028F1D0214608310C4800F074
:10DF200019F870BD0023A0881A46194686DFC9E794
:10DF30000023A0881A461946A9DFC3E721460448F2
:10DF400000F008F970BD0000182600200005005000
:10DF5000B82C002030B5044687B00020059003900F
:10DF600004900090019002900D7B38482B00FDF743
:10DF700019FF076A052D3B236A4E6A004A89062A63
:10DF800001D0032216E042888280487B0190087C01
:10DF90004A7C000412061043CA7B8B7B1102194392
:10DFA0000843029001206946087003AA0020FFF789
:10DFB00093FD024601213CE003206946087003AA54
:10DFC0000020FFF789FD0246042132E04A89032A36
:10DFD00001D0032206E08A7B4B7B1102194341806A
:10DFE00081800122022124E004206946087003AAEE
:10DFF0000020FFF771FD0246012801D0032118E03F
:10E000002046059A049900F075FD07B030BD488997
:10E01000022801D003220BE0487B019006206946CC
:10E02000087003AA0020FFF757FD0246012804D01C
:10E030000621204600F0B8FDE7E703AD0ECD2046EF
:10E0400000F082FDE1E703222946F2E718260020CE
:10E05000FFF706FEBFF34F8F04490348C860BFF3C4
:10E060004F8F00BFFDE700000400FA0500ED00E05F
:10E0700010B5134A00215170017A012911D00229EB
:10E080000ED18189491C8181C189491C89B2C18114
:10E09000028A914204D1002100F006FE00F07AFCD1
:10E0A00010BD838AC28A991AFF2901DC89B201E076
:10E0B000FF210131511889B2C1829942EBD010BDC4
:10E0C0006C26002030B587B000240194029403949C
:10E0D00004948A1D8B790831022B33D153888589AA
:10E0E000AB422FD1127A042A2CD0062A2AD0052A34
:10E0F00028D002236A461371012595720D899581F6
:10E100004D89D5810C310594049193820692104D6E
:10E11000018A05AA2888A5DF002804D16846FEF7F1
:10E120009FF9002807D06846048101A92888A8DF44
:10E1300000280AD006E0FF20FE306946088101A9C8
:10E140002888A8DF002007B030BD0120FBE70000D1
:10E150001826002030B50546C888AA8887B09042A6
:10E1600023D100200590039004900090029002209B
:10E170006A461070084612300190088A029003AA7D
:10E1800069460020FFF7A8FC094C608800280CD0E5
:10E19000A088401E0004000CA08006D12846059AE5
:10E1A000049900F0A7FC6088A08007B030BD000093
:10E1B00018260020F8B50D4614460646694600F0BC
:10E1C00058FA00280DD0009BFF2B09D8581C834219
:10E1D00006D869788909022902D02979814201D2B9
:10E1E0000020F8BD2370611C3046009A00F066FBE9
:10E1F000F8BD10B5114600F0D1F810BD10B51146AC
:10E2000000F0E1F810BDF8B50C4615460646694623
:10E2100000F02FFA00280BD0009A501C904206D331
:10E2200061788909022902D02179814201D2002036
:10E23000F8BD2946304600F041FB009A0021A95460
:10E24000F8BDF0B585B00C468E68174605466946A0
:10E2500000F006FB00280ED0A06800280BD06078E4
:10E260003A468006800F02283146684605D000F005
:10E27000D7F80199696005B0F0BD00F081F8F8E7C2
:10E280007CB50D461446694600F092F900281FD06F
:10E290002879082806D0042808D0022809D00128A7
:10E2A0000BD014E00098019903C40AE000982060A4
:10E2B00006E0009800B2208002E0009840B2207092
:10E2C000C117009A019B50405940084301D00020DB
:10E2D0007CBD01207CBD7CB50D461446694600F02E
:10E2E000A5F900281FD02879082807D00021042884
:10E2F00008D0022809D001280BD013E0009801991A
:10E3000003C409E00098206006E0009880B22080F5
:10E3100002E00098C0B22070009A019B5040594022
:10E32000084301D000207CBD01207CBD7CB50D469A
:10E330001446694600F07AF900281ED02879009921
:10E34000082807D0CA17042809D002280AD00128B3
:10E350000BD011E0019A06C40846134608E00846AF
:10E36000216004E008B2208001E048B22070C317A9
:10E3700048405340184301D000207CBD01207CBDA3
:10E3800070B50D46064614461146284600F083FA3D
:10E3900022462946304600F043F870BD38B50C4699
:10E3A0000422694600F08AFA00280BD0684680787B
:10E3B00001046846C07800060143684600880143AE
:10E3C0000120216038BD1CB50C460822694600F0CA
:10E3D00075FA002823D069460A784978080E0902A0
:10E3E0000A4369468B78190C1B0408431A43694693
:10E3F000CB78190A0843694609791B060843694620
:10E4000049791A430902084369468979090408438E
:10E410006946C979226009060843606001201CBD75
:10E42000F0B5054600209DB001900646029004A874
:10E4300000F058F98BE003AB0AAA6946284600F0C1
:10E44000D2F800280BD004A80A9900F05CF9002843
:10E450000BD0059840788006800F59D066E068465A
:10E46000007B002878D11DB0F0BD0A98B04249D396
:10E47000059C04AE059840780007000F082814D0CA
:10E48000304600F057F90598A042F3D10026F64334
:10E490000A98B04236D3A96811910C90684600786A
:10E4A0000B9008980468169122E005980678EFE72B
:10E4B00020680768002F05D0214628460B9B0C9A40
:10E4C000B84712E0129520680C9980680B9F00787D
:10E4D00088420CD1214617A8FEF7E2FC01212173E6
:10E4E00017AA39461298FEF7F8F80028BBD0A4689E
:10E4F000002C03D0A96816988142D9D0A968119838
:10E50000814224D168460178284600F015FA1CE0C3
:10E51000069840280AD2C006C00E01218140069804
:10E520004009820001A883580B438350EC68002CFB
:10E5300005D06846027804AB28460A99A047684689
:10E54000017804AA2846FEF7C8F800288BD0A868EE
:10E55000002801D06FE7FFE70598069C457804A8DE
:10E5600000F0E8F80028F7D1A806800F04D105983C
:10E570000078002800D0641C002C17D0002001A9CE
:10E58000630904E082008A58521C0DD1401C83426A
:10E59000F8D898000A58E006C00E2021091A002079
:10E5A000C043C840824201D000205CE701205AE706
:10E5B0001CB50C46694600F039F8002812D00098C6
:10E5C000019AC10708D0D10740080843C143520847
:10E5D000D0432160606004E0D1074008084351083F
:10E5E00003C401201CBDF8B5074600201870087050
:10E5F0000E4610601C4615466946384600F039F84C
:10E600000146012000290AD0009900290CD0C80831
:10E61000286000984007400F30700120F8BDB968AD
:10E62000002901D00020F8BD2070FBE7F3B50026DB
:10E6300081B03446354603E0402E01D30020FEBDB4
:10E640006946019800F068F90028F8D06846077814
:10E6500032467806400EC10FFCF774FB2943044391
:10E66000F61D0D463806E7D402980460416001208B
:10E67000FEBDF8B50E460746694600F04DF9002884
:10E680000AD068460478200616D507256406640E6D
:10E6900003E0202D01D30020F8BD6946384600F084
:10E6A0003BF90028F8D0684601784806400EA8409B
:10E6B0000443ED1D0806ECD401203460F8BD0000D1
:10E6C0005968064A8968914206D141688068044ABF
:10E6D000491C401E1160506070470000A0F3030009
:10E6E000FC250020016000238360C26041608B78BC
:10E6F0009A1803230261CB56D21842610878002889
:10E7000000D00120704770B545680E460446606829
:10E710000178B14206D140780007000F082801D0E7
:10E72000012070BD204600F005F86068A842EED1D7
:10E73000002070BD30B541680A78002A0CD00B4625
:10E740000C3343600A7B002A08D04C780A79A5066E
:10E75000AD0F032D07D00BE0002030BDC26801686B
:10E76000FFF7C0FFF8E75D78AD06AD0F032D06D0CB
:10E770002509022D09D0A409022C09D009E08D78C1
:10E7800004690022641B046103E04C79624300E0E9
:10E79000042249788906890F02D18168491C816069
:10E7A0009C78016909198918032201619A56891810
:10E7B0004161012030BD30B541680024497887B0FF
:10E7C0000A07120F082A10D08A091DD08A09022AC6
:10E7D00009D102698906890F1460022901D0032931
:10E7E00001D14069047007B030BD0069056808E0D8
:10E7F0002C7329466846FEF753FB6846FFF7DBFF9C
:10E80000AD68002DF4D1EEE78906890F012911D0FA
:10E810000229E6D00329E4D0426851780907090F9C
:10E8200007290AD0916800290CD012790069FCF7F9
:10E8300099FAD8E741690C70EEE70169906800F039
:10E840002AF8D0E711790069FCF7A5FACBE70000B8
:10E8500010B5024B002408C016C010BDD3C403007D
:10E8600038B50D4604466946FFF703FF00280BD074
:10E87000E368A16805CCEB60A96005C50098083C79
:10E88000083D814201D2002038BDA860A168081A65
:10E89000A060012038BD00B50A4687B00146684631
:10E8A000FFF720FF002807D06846FFF784FF68467F
:10E8B000FFF740FF0028F7D107B000BD7FB5144631
:10E8C0000546002915D1134A2868904208D110E066
:10E8D000102269462846FFF7F1FF002807D0103CB8
:10E8E000102CF5D8224669462846FFF7E7FF04B00A
:10E8F00070BDA868A04201D20020F8E72B6822462C
:10E90000284698470028F2D0A868001BA86001207C
:10E91000EDE70000D3C4030010B50446806800286A
:10E9200009D02368012220469847002803D0A06818
:10E93000401EA060012010BD38B50024002907D07A
:10E94000012913D0022913D005291FD0002038BD7A
:10E950000546012269462846FFF7B0FF002813D07C
:10E96000684600780006F4D4012038BD08220EE085
:10E9700005466946FFF77DFE002805D000212846A0
:10E98000009AFFF79BFF38BD204638BD04220021C6
:10E99000F7E700000848416E491E416604D1074967
:10E9A000FD230A781A400A70016E491C0166042989
:10E9B00001D10021016670478C3100206C260020B7
:10E9C00070B50C490446486E042810D00A6E12181F
:10E9D000042A00D3121F401C4866182042435518D1
:10E9E00001462846FCF7D7F90120256070BD0020BC
:10E9F00070BD00008C31002010B518481822016E3F
:10EA000051430C18406E00281FD0207A012802D0F4
:10EA1000022816D10FE0A18AE08A091AFF2901DC39
:10EA20008AB201E0FF220132E168800023690918FF
:10EA3000181829DF01E0A08928DF112806D0002856
:10EA400003D00921204600F02FF910BD0449FD2212
:10EA50000878104004221043087010BD8C3100204B
:10EA60006C26002010B5054801784A07920F04D1A2
:10EA7000022211430170FFF7BFFF10BD6C2600207A
:10EA8000016806C98A4201D3501A70478068401A4B
:10EA9000401C80187047F8B51E681C46154607468E
:10EAA000002904D0012917D0052921D118E0002020
:10EAB0002060401C2060B0421AD801222946384606
:10EAC000FFF7FCFE002806D028786D1C000601D553
:10EAD0002068EEE70120F8BD08200246186002E039
:10EAE00004200246186029463846FFF7E7FEF8BDC5
:10EAF0000020F8BDF7B5114D0A4606462888104992
:10EB0000884218D0287AC00715D00E4C602020709B
:10EB1000032161700120A070E11C104600F0D2FBBF
:10EB2000C71CE119029800F0CDFBC219B1892888F1
:10EB300000F0DEF8FEBD0820FEBD00001826002013
:10EB4000FFFF0000CC2C0020FFB5144D0A460646FE
:10EB50002888134981B088421ED0287AC0071BD06C
:10EB6000104C60202070062161700120A070E11C13
:10EB7000104600F0A7FBC71CE119039800F0A2FBA8
:10EB8000C719E119049800F09DFBC219B1892888C2
:10EB900000F0AEF805B0F0BD0820FBE71826002015
:10EBA000FFFF0000CC2C002070B50A4B04461888EB
:10EBB000094DA8420CD01B7ADB0709D0074B602512
:10EBC0001D7059709A700322A18900F091F870BDF0
:10EBD000082070BD18260020FFFF0000CC2C00206C
:10EBE00070B501240B49600408600B49401088602F
:10EBF000094940398860094D6C602F20FEF788FA7A
:10EC0000AC60074D00242F20AC60FEF781FAAC7099
:10EC100070BD000080E100E04013014000100140A1
:10EC20004026002010B50446FDF7D8F800280CD087
:10EC3000A007C00E002C0ADA2107090F083989083D
:10EC4000144A89008918C96906E0134810BDA10853
:10EC5000124A890089180968C1400806800F0428F3
:10EC600011D200280FD002280DD00D494B68E206C2
:10EC7000D20E01209040002B08D0620992008B58E0
:10EC800003438B5004E00448401C10BD0549086054
:10EC9000002010BD00ED00E00120000000E400E0D5
:10ECA0006426002000E100E01FB5002200920192DE
:10ECB00002920392037A012B02D0022B11D106E0BB
:10ECC0006B461A7002690292828A9A8109E00123D6
:10ECD0006A4613708289C389D31A6A46138183896D
:10ECE00053814268019200688268684690471FBD60
:10ECF00007B584B00022009201926A46118001217A
:10ED0000917006A90291034903916946A6DF07B0F5
:10ED100000BD0000CC2C0020F8B516460D460400BE
:10ED200008D0002D06D0206C8022002138282254E3
:10ED300003D307E00E20F8BD2154401C3828FBD334
:10ED40000BE02154401C4028FBD32146084600F02C
:10ED500095F838212046FCF71EF8236CA26C590F59
:10ED6000DB00E06CD21848412146A2640306170A72
:10ED70002031E0641F43CA778F770304170C1F43C9
:10ED80000302100E4F7718430877E06CC876020A2A
:10ED90008A76020C4A76000E08762146084600F074
:10EDA0006DF8002E1ED00021E26EC800C2406A54E9
:10EDB000A36EC3406A181371636EC3401372236E4F
:10EDC000C3401373E36DC3401374A36DC340137545
:10EDD000636DC3401376236DC340491C1377042928
:10EDE000E2D31FE000211823C800226D181AC24088
:10EDF0006A54666DC6406A181671A66DC6401672D2
:10EE0000E66DC6401673266EC6401674666EC64022
:10EE10001675A66EC6401676E66EC640491C167775
:10EE20000429E1D30020F8BD002815D00021016499
:10EE30008164C164094901650949416509498165E0
:10EE40000949C1650949016609494166094981665F
:10EE50000949C166002070470E20704767E6096ABD
:10EE600085AE67BB72F36E3C3AF54FA57F520E51EB
:10EE70008C68059BABD9831F19CDE05BF0B5CCB096
:10EE8000002214460CAB0D196E782F7836023E43E3
:10EE9000AF7876BA36043F02ED783E432E439500B4
:10EEA000521C241D5E51102AEDD320E09100CD1894
:10EEB000803DAB6F8C4611241946E14113241E4658
:10EEC000E64171409B0A59406B6C07271E46FB4187
:10EED00034461227FC415C40F3085C4009192C6C55
:10EEE0006B6E1B19CC1861460CAB5C50521C402A4F
:10EEF000DCD3016D0B91476D0A97836D0993C26D49
:10EF000006920092026E0892446E0794A646846EA2
:10EF100005940194C46E049402940024A446062629
:10EF20001446F4410B261546F5416C40192615464A
:10EF3000F5416C40019E7546154096436E40A619FA
:10EF40006446A400254D03942D59029C2C193619B2
:10EF5000039C0CAD2C590D463419039402260C4623
:10EF6000F4410D26F541654016260C46F4416540F6
:10EF70003C465C403E460C401E4074402D19019CAE
:10EF8000029474469646009A0194039C00933B4673
:10EF90000F46121961196446641CA446402CBED366
:10EFA0000B9C611801650A99C91941650999C9182D
:10EFB0008165009B0699C918C16508998918016681
:10EFC000079971444166019A059989188166029AE8
:10EFD00004998918C1664CB0F0BD000084F50300A7
:10EFE000F0B516460F46040005D0002E1ED0002FA7
:10EFF00001D0002518E00E20F0BD216C785D605432
:10F00000206C401C206440280DD121460846FFF7A3
:10F0100035FF0123A16C5B020022E06CC918226459
:10F020005041A164E0646D1CB542E6D30020F0BD00
:10F03000002803D00249C860002070470E207047A6
:10F04000702600201CB5034901910091694660DFDC
:10F050001CBD0000E025002070B50E460546144694
:10F0600014211046FBF797FE01200021208021612A
:10F07000217326726572002D00D0A072002070BD31
:10F0800010B5002902D00020FCF716FFFDF78EFE18
:10F0900010BD000010B50021024A0846FCF70EFF23
:10F0A00010BD000081F0030010B5FCF703FF10BD98
:10F0B000F8B5002903D08C070025002C01D00720CB
:10F0C000F8BD0E4E0E4FB160728073603968012436
:10F0D0006603314203D00A49254680310E60094952
:10F0E00010DF002803D0002DEAD03E60F8BD0348B1
:10F0F00004701620FFF796FDF8BD00007026002072
:10F1000000E100E0A9F0030001480078704700002A
:10F1100070260020002803D00249086100207047B3
:10F120000E20704770260020FEB51F4C0025A768F2
:10F13000606802906846FDF70BFD0190FDF7C6FE82
:10F1400006460198002822D000230098616817E045
:10F150000E680A46864202D9301A086012E0801B07
:10F16000F31800261660D668D169B446002E07D081
:10F17000FE183602360A566066469660D561154618
:10F180000029E5D128466160FDF7F6FE06E0284635
:10F19000FDF7F2FE002801D1002E02D00298FDF703
:10F1A000B7F90020E070FEBD402600200120024992
:10F1B000000508607047000000E200E010B50E4B4B
:10F1C0005968002906D002680C68A24204D8A21A25
:10F1D0000A60C161586010BD0B4604E00B46C96966
:10F1E000121B002904D00C689442F7D3A41A0C60B7
:10F1F0000260C161D86110BD402600207CB50D467B
:10F200000646002469460C706846FCF79BFF01A87F
:10F2100000F094F800280DD0057046606846084953
:10F220000079487068460078FCF7AAFFFFF7BEFF38
:10F2300020467CBD684604240078FCF7A1FFF7E770
:10F2400050260020F8B51D4D6C68002C34D01C48A9
:10F2500000274068A968401A0602360A2068B042B2
:10F2600018D8361AC7192246107CE46900280FD036
:10F2700000201074EB68002B07D091695069984703
:10F28000002805D0FCF718FE02E051699069884714
:10F29000002CE3D129786878814206D1401CC0B2A5
:10F2A0006870022801D10020687004490006800DB2
:10F2B00018310F50FFF77AFFF8BD000040260020FC
:10F2C000001501400870020A4A70020C8A70000E94
:10F2D000C87004207047000038B51549154A4888A1
:10F2E00090420FD04A78144C521CD2B24A70237B01
:10F2F000934208D3091D75DF002803D0A1690029B6
:10F3000000D0884738BD00254D70217C002907D0EA
:10F310003B2176DF002803D0A169002900D088476F
:10F3200061690029EED068460570884738BD000045
:10F3300004260020FFFF0000542C002010B50949CE
:10F340004B788C785A1CD2B2944200D100220C78AF
:10F35000944201D1002010BD0270486818214B432F
:10F36000C01810BD5026002010B501E0FDF736FA98
:10F37000FDF76CFC0028F9D110BD00000101000070
:10F380000100000000000000020500002100000054
:10F39000000000000000000000000000000000006D
:10F3A000011104FC0400000000000000021104FC34
:10F3B0000400000000000000032104FC040400001D
:10F3C00000000000041101FF010000000000000027
:10F3D000051102FE0400000000000000061104FCFC
:10F3E0000400000000000000071104FC04000000FD
:10F3F00000000000081701FF220000007CF303005A
:10F40000091001FF010000007AF303000000000072
:10F4100000000000000000000101000004000000E6
:10F4200000000000000000000000000000000000DC
:10F43000011101FF0100000000000000021702FEA0
:10F4400064000000A0F30300031704FC04000000A4
:10F4500018F403000000000000000000000000009D
:10F46000010700007000000030F4030002010000FA
:10F470000100000000000000030500004100000042
:10F48000000000000000000000000000000000007C
:10F49000011704FC7000000030F40300021704FCA4
:10F4A000B400000060F40300000000000000000051
:10F4B00000000000CF3F998E73EBCA98FE897B5104
:10F4C000A5E555658CE600777A1E7CD28DA4B871CF
:10F4D0000BAE51180822E3C7190C0E58A0DDE3BC8F
:10F4E000B5F7196FFEC0C1F88D347BB3F206FE96F6
:10F4F0006C215E55B4F40300400000001516171887
:10F5000011121314342C00200200000750EADA30E4
:10F510008883B89F604F15F30000C98E010000007A
:10F5200000000000000000000000000001000000DA
:10F5300000000000000000000000000002000000C9
:10F5400000000000000000000000000003000000B8
:10F5500000000000000000000000000004000000A7
:10F560000000000000000000000000000003000098
:10F57000803100205C3100202000000001000000EC
:10F5800000000000982F8A4291443771CFFBC0B52C
:10F59000A5DBB5E95BC25639F111F159A4823F925E
:10F5A000D55E1CAB98AA07D8015B8312BE853124B7
:10F5B000C37D0C55745DBE72FEB1DE80A706DC9B78
:10F5C00074F19BC1C1699BE48647BEEFC69DC10F24
:10F5D000CCA10C246F2CE92DAA84744ADCA9B05C60
:10F5E000DA88F97652513E986DC631A8C82703B023
:10F5F000C77F59BFF30BE0C64791A7D55163CA0631
:10F6000067292914850AB72738211B2EFC6D2C4D3C
:10F61000130D385354730A65BB0A6A762EC9C2812A
:10F62000852C7292A1E8BFA24B661AA8708B4BC2C0
:10F63000A3516CC719E892D1240699D685350EF4EA
:10F6400070A06A1016C1A419086C371E4C774827A1
:10F65000B5BCB034B30C1C394AAAD84E4FCA9C5B17
:10F66000F36F2E68EE828F746F63A5781478C88468
:10F670000802C78CFAFFBE90EB6C50A4F7A3F9BE4A
:10F68000F27871C62DE30300D7E2030081E20300A4
:10F69000F3E10300FDE10300B5E1030007E203002D
:10F6A00043E203000000000008200001FFFFFFFF0D
:10F6B000FFFFFFFFFFFFFFFF000000000000000052
:10F6C0000000000001000000FFFFFFFF512563FC68
:10F6D000C2CAB9F3849E17A7ADFAE6BCFFFFFFFFCD
:10F6E000FFFFFFFF00000000FFFFFFFF96C298D85A
:10F6F0004539A1F4A033EB2D817D0377F240A4635B
:10F70000E5E6BCF847422CE1F2D1176BF551BF3763
:10F710006840B6CBCE5E316B5733CE2B169E0F7C36
:10F720004AEBE78E9B7F1AFEE242E34F4B60D22703
:10F730003E3CCE3BF6B053CCB0061D65BC869876F9
:10F7400055BDEBB3E7933AAAD835C65A91AF03003B
:10F75000A5BB0300B1B9030080F70300E02500203A
:10F76000B8000000BEBD030038F803009826002052
:10F77000A0110000CEBD030085C3030005C3030034
:10F780000100000000000000000000000000000078
:10F790000000000000000000000000000000000069
:10F7A0000000000000000000000000000000000059
:10F7B0000000000000000000FFFF0000000000004B
:10F7C0000000000000000000000000000000000039
:10F7D0000000000000000000000000000000000029
:10F7E0000000000000000000000000000000000019
:10F7F0000000000000000000000000000000000009
:10F8000000000000000000000000000000000000F8
:10F8100000000000000000000000000000000000E8
:10F82000000000000024F40000100000000C0400A0
:08F830000DCC030000000000F4
:020000041000EA
:0410140000AC030029
:040000050003ACC187
:00000001FF
